:03000000020053A8
:0C005300787FE4F6D8FD7581200200667D
:10024C00D2B07F3212025EC2B0AF0312025ED2B0E5
:02025C007F32EF
:09025E001FEF6004000080F8228B
:100267007D997C03000000ED1D70011C144C70F794
:09027700EF1F70011E144E70E728
:01028000225B
:0602180012021E12021E7C
:10021E00E4F509F50AF58AF58C30B4FDD28C20B4DC
:10022E00FDC28CAF8C7509008F0AE50A750A00F5C0
:0E023E0009AF8AEF250AF50AE43509F5092211
:02019E00AB07AD
:1001A000EB75F00584F9E4FAEAC399505CC2B2C277
:1001B000B17F027E00120267D2B312024CC2B0AF0E
:1001C0000312025E12024CC2B3C2B07F027E001262
:1001D0000267D2B2D2B17F3212025EC2B1AF031255
:1001E000025ED2B17F3212025EC2B1AF0312025E72
:1001F000D2B17F3212025EC2B1AF0312025ED2B13F
:100200007F3212025E0A0201A8C2B2C2B1C2B3C2F8
:08021000B07F057E00020267C9
:10006600C2B0C2B1C2B2C2B375B20F7F907E0112E6
:1000760002677FC812019E7F9612019E7F6412015D
:100086009E7F587E021202677589011202181202BB
:100096001E12021E12021EC3E50A94BEE50994054D
:1000A60040F2D3E50A94FAE509940550E77F641215
:1000B600019E7F9612019E7FC812019E75A88075CB
:1000C600AF0475D7F675D6FF758E1012021E120292
:1000D6001E12021E12021E30020A7F327E00120219
:1000E60067120218D3E50A94F4E509940140E2E5A3
:1000F6000A94C4E509940950D8E4F50DF50EC20238
:10010600C3E50A94FAE5099405401CE50A2410FFA4
:10011600E50934FAFEEF7802CEC313CE13D8F9F50B
:100126000FC201D2008031D3E50A94BEE5099405D9
:10013600501DC374C8950AFF74059509FEEF780231
:10014600CEC313CE13D8F9F50FD201D2008009E43D
:10015600F50BF50CC2B2C2B32000030200D7C200F1
:10016600A201300301B3500FE4F50BF50CC2B2C285
:10017600B37F03FE120267A201920330010DD2B2D1
:10018600C2B3E4F50B850F0C0200D7D2B3C2B2E4BA
:08019600F50C850F0B0200D7E8
:0300630002000395
:10000300C0E0C0D00508E50864647025F508050E56
:10001300E50E7002050DD394F4E50D9401401275BD
:100023000D00750E00D202750B00750C00C2B2C232
:10003300B3E50BD395084004D2B08002C2B0E50CFF
:10004300D395084004D2B18002C2B1D0D0D0E032FF
:00000001FF
